:020000040000FA
:10000000073099008316FF2390000A308500831281
:100010008501B121850185181428D321D3218518A4
:1000200014280000C12113288501A9013F30A9002F
:10003000AB01AA21AB00FF302B020319DB280130F2
:100040002B020319F92802302B0203191729033058
:100050002B020319352904302B02031953290530CB
:100060002B02031971294528000000000000000040
:10007000000000000000000000000000000000344C
:1000800085163420851234200800A901AA01083001
:10009000AA000030A9000516342034204020342066
:1000A000342005128F21AA21A90A03110310250665
:1000B000031D5D28AA0B5228D828A901AA010830DF
:1000C000AA000830A900051634203420402034202E
:1000D000342005128F21AA21A90A03110310250635
:1000E000031D7528AA0B6A28D828A901AA0108307F
:1000F000AA001030A90005163420342040203420F6
:10010000342005128F21AA21A90A03110310250604
:10011000031D8D28AA0B8228D828A901AA0108301E
:10012000AA001830A90005163420342040203420BD
:10013000342005128F21AA21A90A031103102506D4
:10014000031DA528AA0B9A28D828A901AA010830BE
:10015000AA002030A9000516342034204020342085
:10016000342005128F21AA21A90A031103102506A4
:10017000031DBD28AA0BB228D828A901AA0108305E
:10018000AA002830A900051634203420402034204D
:10019000342005128F21AA21A90A03110310250674
:1001A000031DD528AA0BCA28D828051105104528F3
:1001B0000515051445283F30A9000130A5009B21F5
:1001C000E2204528051634203420402034203420F5
:1001D0000512A801A9010030A9000830A8008F214C
:1001E0009B21A90AA80BEF28A8010130A800CA2169
:1001F00008003F30A9000230A5009B2100214528BE
:100200000516342034204020342034200512A80163
:10021000A9010830A9000830A8008F219B21A90A54
:10022000A80B0D29A8010230A800CA2108003F3000
:10023000A9000330A5009B211E2145280516342066
:1002400034204020342034200512A801A9011030A8
:10025000A9000830A8008F219B21A90AA80B2B29EF
:10026000A8010330A800CA2108003F30A9000430CB
:10027000A5009B213C214528051634203420402030
:10028000342034200512A801A9011830A900083033
:10029000A8008F219B21A90AA80B4929A801043095
:1002A000A800CA2108003F30A9000530A5009B2105
:1002B0005A2145280516342034204020342034208B
:1002C0000512A801A9012030A9000830A8008F213B
:1002D0009B21A90AA80B6729A8010530A800CA21FB
:1002E00008003F30A9000630A5009B217821452851
:1002F0000516342034204020342034200512A80173
:10030000A9012830A9000830A8008F219B21A90A43
:10031000A80B8529A8010630A800CA2108000830CA
:10032000A700A5016400031085192514A50D402020
:10033000A70B93290034290883169B0025089A00EF
:100340001C1555309D00AA309D009C149C18A629B0
:1003500083120800290883169B001C141A088312B4
:1003600008000730A0002F30A1000330A200A00B2E
:10037000BA29A10BBC29A20BB729BE29BF29C029C4
:100380000800A9013F30A900FF30A5009B21A8016A
:100390000330A80005150514B12105110510B12180
:1003A000A80BCA29080064005030AC00AD0BD62958
:0603B000AC0BD62900345D
:02400E00443F2D
:00000001FF
